:020000000F28C7
:10000800FE00030EF1000408F2000A08F300831250
:100018007F08F4007D28B3288B01073083129900EC
:10002800703083169F0006309100493083129F007C
:1000380085010630831685008312870101308316F7
:100048008700843081007D30F5007508FC00FA01D6
:100058007D30F5007508FB00F601F901F701F8019C
:100068000630831281008B168B17FB08031D392875
:100078007A307902031C442886307902031C482808
:100088000130F5007508F7077A307902031C51280A
:100098008630790203185128F70183120718582867
:1000A80003307702031C5D28FA30F5007508F60066
:1000B800F801F608031907186728033077020318B0
:1000C8006728F801F80AF808031D6C2887106D28BE
:1000D8008714F930F5000000F50B6F28732800002D
:1000E80083129F149F1876281E08F5007508F900DA
:1000F80039280B1DA8280B11063081000130FC029D
:10010800FC08031D96287D30F0007008FC000430C0
:10011800F0007008FA00F808031D952820308706BB
:10012800962887167A0803199D280130FA020716BF
:100138009E2807127B080319A3280130FB027608C2
:100148000319A8280130F6027408FF0073088A0012
:1001580072088400710E8300FE0E7E0E0900F601FF
:0C016800F701F801F901FA0183011028E9
:02400E00E1F3DC
:00000001FF
